:020000040000FA
:02000000522884
:080008000000F800030E830163
:10001000F9000A08FA008A010408FB00831203139E
:10002000101083120313FC03031D1E2818308E00CA
:1000300080308F002030FC00FD0A2228C5308E0061
:1000400066308F00831203130C10831603130C14F5
:10005000831203131014831203137B0884007A089D
:100060008A00790E8300F80E780E090083120313BC
:100070000B178B17831203130030831203132030E6
:10008000FC00831203130C10831603130C14831249
:10009000031310148312031308000030B50010304E
:1000A000B6000800A101FD01A001B7012F21D22057
:1000B0007D244D20FC20AB01F6243620DC25452292
:1000C000211B93202119F62441084202031DDC2440
:1000D000A11944258B216A2336088A00350882003D
:1000E00000308A00FF30B300A11A022521187F28B2
:1000F000A601A60300000000031D79285F282B0835
:10010000A400A721B623D823DF230D254108FF3CF7
:10011000031D5F282B08A400A721B623D1234C245C
:10012000122521105F2821135D08023C0319B52810
:100130005D08013C0319A5285D08033C0319A428A8
:10014000043C0319B428080083172A0884006008B7
:100150008000840A61088000840A62088000840AA2
:10016000630880008313080008002B08A400EC201B
:10017000A20AF420A6012608603E84000008DF00E1
:1001800083172A087F39260784005F0880008313BD
:10019000A3006E21A20AA60A2608043C031DBB2860
:1001A000A7210800831203138501860187018801B6
:1001B00089018316031306309F00FC308500F03060
:1001C000860081138701FF30880000308900C0302D
:1001D0008B008312031308002408A2000310A20D51
:1001E000A20DA20DA20708002408AA000310AA0D60
:1001F000AA0DA030AA070800A401EC20F4202408CE
:10020000E03E840083175D218000A20A2A087F391E
:1002100084005D218000A20A840A5D218000A20A78
:10022000840A5D218000A20A840A5D218000831374
:10023000A20A2A0884005D218000A20A840A5D21A6
:100240008000A20A840A5D218000A20A840A5D213E
:100250008000A40A2408103C031DFD280800FE307D
:10026000A2005D21A5302302031D3C29A20A5D21C5
:100270005A30230203190800A201A401A501250890
:100280008A150A168027A30001308A006E21A20A6F
:10029000A50A2508093C031D3F29A501A40A240835
:1002A000103C031D3F29FE30A200A530A3006E21A3
:1002B000A20A5A30A3006E210800831203132208F9
:1002C000831203178D00831603178C130C148312EB
:1002D00003170C0883120313A300080083120313EF
:1002E0002208831203178D0083120313230883123D
:1002F00003178C00831603178C130C158B135530C2
:100300008D00AA308D008C148B178C1885290C1148
:100310008312031308007D08211E9029A000080005
:10032000200203190800A00A01308506A401A721B4
:10033000AC1FA0292C1F9E29EA219F29BE211C2227
:10034000A40A10302402031D972921140800240850
:10035000E03E840083170008AC00F4202A087F39AF
:1003600084000008AD00840A0008AE00840A00087A
:10037000AF00840A0008B000831308002A08840034
:10038000800A031DCD29840A800A031DCD29840A11
:10039000800A031DCD29840A800A2A0884000008E7
:1003A0002D02031D0800840A00082E02031D080008
:1003B000840A00082F02031D0800840A0008300286
:1003C000031D0800800184038001840380018403ED
:1003D000800108002A0884008008031D062A840A78
:1003E0008008031D062A840A8008031D062A840A41
:1003F0008008031D062A3008800084032F0880002F
:1004000084032E08800084032D0880002A088400BD
:100410008003FF300002031D0800840A8003FF30C0
:100420000002031D0800840A8003FF300002031D40
:100430000800840A800308000430A6002A0884000B
:100440008317000883130002031D0800840AA60313
:10045000031D202A2C080339B100B201AC1D372A34
:100460002408E03E840083178030800683132C1E0E
:100470000800F4202A08840001308000840A8001EA
:10048000840A8001840A80010800013031020319C6
:10049000532A023031020319572A0330310203195B
:1004A0005B2AB10108008A110A12C425512A8A1157
:1004B0000A12D525512A8A110A12DC25512AA600D2
:1004C0002B08E03E8400831726088006831308006B
:1004D0003808E0003908E1003A08E2003B08E30090
:1004E0003C08E4003D08E500080084000730D8001F
:1004F0008001840AD803031D782A080084000308B9
:10050000D900D80159088300800D0308D900840A56
:10051000D80A07305802031D822A080084000630DA
:1005200084070308D900D80159088300800C030808
:10053000D9008403D80A07305802031D942A080002
:10054000D8015808573C84000008DA005808493C94
:1005500084000008DA02031D0800D80A0730580298
:10056000031DA12A080084000730D800800A031D5B
:100570000800840AD803031DB62A08000310D90115
:10058000D801DA015918DA0AD90143305807840032
:100590000008DA070318591451305807840000087E
:1005A000DA07031859145A088000D80A073058028D
:1005B000031DC12A0800D80159145B145130580793
:1005C00084000008DA004330580784000008DA028B
:1005D000031C5B105918F02A0130DA02031C5B106F
:1005E0005130580784005A08800059145B1C591078
:1005F000D80A07305802031DDD2A591C03100800D1
:10060000513075223930DC00DC03031908004A1828
:10061000BE2203104A308E22031043307E22042B68
:100620004A3075223830DC00C91B1E2B43300310C2
:100630007E22DC03031D142B03150800A0220308EF
:10064000DB004A307E225B0883000318DB220311A3
:10065000031043308E22DC0A39305C02031D1E2B4E
:1006600008004A08D1004B08D2004C08D3004D08BE
:10067000D4004E08D5004F08D6005008D700080017
:100680005108CA005208CB005308CC005408CD00D2
:100690005508CE005608CF005708D0000800510872
:1006A000E0005208E1005308E2005408E300550856
:1006B000E4005608E50008006008C3006108C400B3
:1006C0006208C5006308C6006408C7006508C80062
:1006D000C90108000130A400FF3024068600033061
:1006E000A600A603031D712BF0300605F03A031D8A
:1006F000802B0310A40D0F30A405031D6C2B992B28
:10070000A500A50EB40124089E230319972BB4005D
:100710000310B40D0310B40D25089E230319972B65
:10072000B4063408A11CB300A11403110800FE3064
:100730009B2BA110FF30B40003150800A6000F305A
:10074000A605A7010130A800280826020319B32B2B
:10075000A70A0F3028050319B02B0310A80DA42BEE
:10076000FF300315080027080311080051307522D7
:10077000433075222A0884000008D400840A000847
:10078000D500840A0008D600840A0008D700831325
:100790002D08C3002E08C4002F08C5003008C6006D
:1007A000102B3123433075228030C500BE22402BF0
:1007B000433075224630C4000530C500002B0A3096
:1007C000B800BA00BC000630B900BB00BD00433021
:1007D00075220430C60010233830A4003123433082
:1007E0007522240884000008C30010232408840014
:1007F00051088000A40A3E302402031DEE2B08009D
:100800000A30B800BA00BC000630B900BB004A305C
:1008100075220430A4006508CA00433075223830C0
:10082000240784000008C30000234A30752260308A
:10083000240784000008C300BE224023A403FF3025
:100840002402031D0D2C433075220430C300002305
:100850005130B3225130B32208005408D700530856
:10086000D6005208D5005108D400D301D201D101DD
:10087000433075224630C4000530C50010230800FF
:10088000433075222D08C3002E08C4002F08C50070
:100890003008C60000230800CD01CE01CF01D001F1
:1008A000433075220A30C30000235408BD00D40130
:1008B00040230A30C30000235408BC00D401402365
:1008C0000A30C30000235408BB00D40140230A307F
:1008D000C30000235408BA00D40140230A30C300E7
:1008E00000235408B900D40140230A30C300002378
:1008F0005408B800D40140230800D324D324D324BF
:10090000D324D324D3240030890030308700BF247F
:10091000D324D324D324D324D32438308700BF2432
:10092000D324D324D324D324D32438308700BF2422
:10093000D324D324D324D324D32438308700BF2412
:1009400008308700BF2401308700BF2406308700AD
:10095000BF2408308700BF2402308700BF24091459
:100960000C30BA24FF30C100C2000800870009140F
:10097000BF24080087000910BF24091408000000E4
:100980000000000000000000000000000000091549
:100990000000000000000000000000000000000057
:1009A0000911D32408001030A4000130A600A60BC2
:1009B000DA2CA40BD72C0800C030BA241030A500C4
:1009C0004108C200FF3C0319EF2C410876258E2513
:1009D0000319EF2CB624A503031DE72C08002030D3
:1009E000B624A503031DEF2CA11608000230BA247B
:1009F0005430B6246D30B62441302B07B624211173
:100A0000A1160800A112B71F0A2D3708BA240E300C
:100A1000BA2408000C30BA240800A1162110843032
:100A2000BA242D2DA116C430BA24162D3030B62488
:100A30002E30B6243D08303EB6243C08303EB62465
:100A40003B08303EB6243A08303EB6243908303EE2
:100A5000B6243808303EB62408003D08303EB6249F
:100A60003C08303EB6243A30B6243B08303EB6242B
:100A70003A08303EB6243A30B6243908303EB6241F
:100A80003808303EB6240800A111C430BA245F2DC6
:100A90003030B6242E30B6246508303EB6246408C3
:100AA000303EB6246308303EB6246208303EB62499
:100AB0006108303EB6246008303EB6240800650860
:100AC000303EB6246408303EB6243A30B62463087B
:100AD000303EB6246208303EB6243A30B62461086F
:100AE000303EB6246008303EB62408008312031757
:100AF0008D0018308F00831603178C170C1400001C
:100B00000000831203170C0883120313BE00831224
:100B100003170E0883120313BF0008003E08831258
:100B200003178D00831203133F08831203178F00EE
:100B3000831603178C170C14000000008312031394
:100B4000BF1BB12D831203170E0883120313C000BD
:100B5000831203170C0D83120313C00DBF17400837
:100B60000800831203170C0883120313C000C0137C
:100B7000BE0A0319BF0ABF13400808000F30A600C1
:100B8000A603031DC02D0800FF30A8002030A700D9
:100B90008A110A12BE25A703031DC82D023085063F
:100BA000A803031DC62D851008001030A900C42518
:100BB000A903031DD72D0800A801C0302808383E1E
:100BC000A7008A110A12BE25A703031DE12D0230DA
:0A0BD0008506A803031DDE2D0800B2
:10200000B701FF30C1000E303302031916280D301E
:10201000330203191E280C303302031D132810301D
:10202000B6002630B5008A110A127028AB0A0F30AC
:10203000AB05211521148A110A127028AB030F3049
:10204000AB05211521148A110A127028B70100303E
:10205000C1000F303302031D31281030B6000030AC
:10206000B5000E303302031D39281030B600E730BA
:10207000B5000D303302031D41281030B600E730A3
:10208000B5000C303302031D49281030B600623011
:10209000B500003033020319542804303302031909
:1020A0005B288A110A12702880308A110A125F2276
:1020B0008A110A12702840308A110A125F228A118E
:1020C0000A1270280130C1000F303302031D6C2842
:1020D0001030B6002630B5000E303302031D7428D0
:1020E0001030B6008730B5000D303302031D7C2858
:1020F0001030B600AC30B5000C303302031D84281C
:102100001030B600D130B5008A110A12702807309D
:10211000C1000F303302031D91281030B600263065
:10212000B5000E303302031D99281030B600AC30D4
:10213000B5000D303302031DA1281030B600623007
:10214000B5000C303302031DA9281130B6001A3037
:10215000B5008A110A1270280430C1000F30330212
:10216000031DB6281030B6002630B5000E303302FD
:10217000031DBE281030B6006230B5000D303302AA
:10218000031DC6281030B6008730B5000C3033026E
:10219000031DCE281030B600DC30B5008A110A12BB
:1021A00070280630C1000130DD001330B600523017
:1021B000B5008A110A1270280630C1000230DD0015
:1021C0001330B600D130B5008A110A1270280230DF
:1021D000C1000F303302031DF1281030B60000306B
:1021E000B5000E303302031DF9281030B60026303A
:1021F000B5000D303302031D01291030B600263022
:10220000B5000030330203190C29043033020319DE
:102210000C298A110A1270281030A1068A110A129C
:1022200070281030A105FC0AFC0AFC0AFC0A8A117D
:102230000A1270280830C1000F303302031D242910
:102240001030B6008730B5000E303302031D2C2944
:102250001130B6006230B5000D303302031D342951
:102260001130B6008730B5000C303302031D3C2915
:102270001130B6003F30B5008A110A1270280630BE
:10228000C1000330DD002B08A4008A110A12A72127
:1022900051308A110A12752243308A110A127522AE
:1022A00083178A110A12BA2383138A110A12D823B8
:1022B0008A110A12DF231330B6005230B5008A119A
:1022C0000A1270280930C1000F303302031D6C2937
:1022D0001030B6008730B5000E303302031D74296C
:1022E0001130B6008730B5000D303302031D7C2954
:1022F0001130B6001A30B5000C303302031D8429AA
:102300001130B600AC30B5008A110A1270280A30BC
:10231000C1000F303302031D91291030B600873001
:10232000B5000E303302031D99291130B6001A3062
:10233000B5000D303302031DA1291130B600623003
:10234000B5000C303302031DA9291230B6007B30D2
:10235000B5008A110A12702803302C05A600031D4F
:10236000B8291230B6004D30B5008A110A12702813
:1023700001302602031DC3291130B600D830B50044
:102380008A110A12702802302602031DCE2911304C
:10239000B600FF30B5008A110A1270281230B6005C
:1023A0002630B5008A110A1270288A110A12702884
:1023B0000B30C100013046230C303302031DE429E9
:1023C0001130B6006230B5000F303302031DEC2926
:1023D0001130B6006230B5000E303302031DF4290F
:1023E0001130B600FF30B5000D303302031DFC295B
:1023F0001230B6004D30B5008A110A1270280C3028
:10240000C100023046230C303302031D0B2A113069
:10241000B6006230B5000F303302031D132A1130AD
:10242000B6006230B5000E303302031D1B2A123095
:10243000B6002630B5000D303302031D232A1130BB
:10244000B600D830B5008A110A1270280D30C100CC
:10245000033046230C303302031D322A1130B600FC
:102460006230B5000F303302031D3A2A1130B60036
:102470006230B5000E303302031D422A1230B6001E
:102480004D30B5000D303302031D4A2A1130B6001D
:10249000FF30B5008A110A1270280E30C1000030DA
:1024A00046230C303302031D592A1130B600623026
:1024B000B5000F303302031D612A1130B6006230BF
:1024C000B5000E303302031D692A1130B600D83032
:1024D000B5000D303302031D712A1230B6002630CC
:1024E000B5008A110A1270282B08E03E8400831779
:1024F0008011001208002C1E8D2AAC1D862A133074
:10250000B6001B30B5008A110A1270281230B600CE
:10251000C730B5008A110A127028AC1D962A1230F5
:10252000B600F130B5008A110A1270281230B600D8
:102530009D30B5008A110A1270280F30C1002B0897
:10254000742200088313AC000C303302031DAC2A44
:102550001130B6008730B5000F303302031DB42AA6
:102560001130B6008730B5000E303302031DBC2A8F
:102570001230B600C730B5000D303302031DC42A37
:102580001330B6001B30B5008A110A1270281030C3
:10259000C1007422001600088313AC000C30330213
:1025A000031DD62A1130B6008730B5000F30330234
:1025B000031DDE2A1130B6008730B5000E3033021D
:1025C000031DE62A1230B600F130B5000D3033029B
:1025D000031DEE2A1230B6009D30B5008A110A1292
:1025E00070281130C1007422801500088313AC00DC
:1025F0000C303302031D002B1130B6008730B500BC
:102600000F303302031D082B1130B6008730B500A0
:102610000E303302031D102B1330B6001B30B500F3
:102620000D303302031D182B1230B600C730B50031
:102630008A110A1270281230C10074228015001607
:1026400000088313AC000C303302031D2B2B113018
:10265000B6008730B5000F303302031D332B113025
:10266000B6008730B5000E303302031D3B2B12300D
:10267000B6009D30B5000D303302031D432B1230E0
:10268000B600F130B5008A110A127028A600E030B9
:1026900084002B0884078317FC30800526088004FB
:1026A00083130800DE018A110A126822A115C430C2
:1026B000B700A1161330B6006130B5008A110A12B6
:1026C00070288A110A160F303302031D6B2B13304A
:1026D000B600B230B5000C303302031D732B13303B
:1026E000B6009930B500B31B962B33080F398A1505
:1026F0000A168E27A6008A110A16A61F822B8A1197
:102700000A1270285E08653C840026080F39800094
:10271000A115DE0A5E088A150A16A327B7008A11DA
:102720000A16A1165E08063C0319992B8A110A1293
:1027300070288A110A162B08A4008A110A12A721F0
:102740008A110A1200248A110A122D248A110A12EF
:1027500040245408E0005508E1005608E2005708FC
:10276000E30021178A110A16B701A1165D08033C80
:102770000319C12B1030B6006230B5008A110A125D
:1027800070281130B6001A30B5008A110A1270286C
:102790000430DD001330B600D130B5008A110A12C2
:1027A000702851308A110A1275228A110A124F2399
:1027B000DE01C43EB700A116A1111330B600E4300B
:1027C000B5008A110A1270288A110A160F303302D6
:1027D000031DEE2B1430B6003830B5000C30330238
:1027E000031DF62B1430B6003730B5008A110A16D7
:1027F000B31B342C33080F398A150A168E27DF00D5
:102800008A110A16DF1F072C8A110A1270284A3013
:102810008A110A1275220A30CA008A110A125C2330
:102820008A110A12002343308A110A1275225F08A6
:10283000C3008A110A12BE228A110A124F235E08AF
:10284000C43E8A110A12BA245F08303E8A110A1265
:10285000B624DE0A5E08C43EB700A1168A110A1625
:102860005E080A3C0319DE038A110A127028211738
:10287000B701A1161030B600AC30B5008A110A12AB
:022880007028BE
:1030000013181A18201827182E1837183D184018AA
:1030100046184C1853185A18611868186F18771802
:103020007E1886188D18E4207535F4395410ED3467
:10303000F2320000E529203A692AE536003900001D
:10304000E4207535F43943106F36EB310000682AFF
:10305000F232AE365310F432F03A0000E529203A4D
:10306000F921EC31A03265266737683A0000E5297E
:10307000203A6F236D39F4300000E529003A000052
:10308000E529203AEC20F23080360000EC20F230C6
:10309000A036692AE5360000EC20F230A036EF2990
:1030A000EE3A00320000EC20F230A036E320693A1C
:1030B000EE370000E529203A6F3A201D69280038D4
:1030C0000000E529203A6F3A201D6528F032000003
:1030D000E529203A6F3A201DE82BF0340000E5295D
:1030E000203A6F3A201DE929653674370000E32045
:1030F000693AEE37201D6F2765370000E320693AF3
:10310000EE37201D6529E539003A0000E320693AD1
:10311000EE37201DF429F0370000E320693AEE373E
:0C312000201DF429F037D215F43900000E
:103F0000A6001F308A002608820780340034463419
:103F1000053400340034003400340034A6001F306F
:103F20008A00260882070034013402340334043442
:103F300005340634073408340934FF34FF34FF34C1
:103F4000FF34FF34FF34A6001F308A0026088207A2
:0E3F5000C434C534C734C834CA34CB34CC347E
:02400E00723FFF
:00000001FF
